:020000040000FA
:04000000000065296E
:040004000034003490
:080008008B13F000030E8301CD
:10001000F2000A08F1008A018C1811288C1AF428C1
:10002000E5288C1051185E29ED1B3B2887184328C2
:10003000D30B5E296C08D6006808EC005608E8006F
:100040006B08D6006708EB005608E7006A08D60080
:100050006608EA005608E6006908D6006508E90067
:100060005608E500E517E917ED171430D300501CCA
:100070005E2951145E29871C4028D30B5E29ED139D
:100080001430D3005E291430D3005C08D600F03958
:10009000DC00D60C560C0339DC0707080C39DC07EA
:1000A0005C080F39D60000308A005608820767289E
:1000B00070286B2867286B286728672870287028A5
:1000C000672867286B2867286B2870286728DE0850
:1000D000031DDE035E29DD0B5E290430DD00A5284B
:1000E000DD0A5D08073C03185E290430DD0078282E
:1000F000DE08031D8C282530EC076C080F39093CFD
:10010000031884280630EC076C08F039903C031C77
:100110008A28E128A030EC02EB0A6B080F39093C71
:100120000318E1280A30EB02EA0A6A080F39093C91
:100130000318E1280630EA076A08F039903C0318F2
:10014000E1289030EA02E90AE128DE08031DB6281A
:100150006C08253C0319D8286C08503C0319DB288F
:100160006C08753C0319DE287530EC006B080F39FC
:100170000319BC28EB03E1280930EB006A080F39AA
:100180000319C428EA03E1286A08F0390319CD28C5
:10019000093EEA001030EA02E1289930EA00E90855
:1001A0000F390319D528E903E1280930E900E128CE
:1001B0000030EC00E1282530EC00E1285030EC0064
:1001C000E128FF30DE00E9175E29D40BEC28831606
:1001D0000C128312D4015E29051EE728D50A5508A2
:1001E0008400000899005E291A08BC008C123B1894
:1001F0004F29BA1B222930088400310884070008DF
:100200003C02031D0D29B10A05303102031D0E29E0
:10021000B101B901FF30BA005E29B101380884008C
:100220003908840700083C02031D2029B90A05305B
:100230003902031D5E29B101B901FF30BA005E2900
:10024000B9015E293C08BA00FF30BB0001308A00CA
:100250003A080F393921CD004D0803193729BD015E
:10026000CE01CD1F5E29CD132808CE005E29D217FE
:100270005E29D70001308A0057080F398207003401
:10028000003480340134003400340034003400344D
:100290000534013400340034003400340034CE0816
:1002A00003195429CE035E29400884003D088407C1
:1002B0003C088000BD0ACD0B5E29D21771088A0068
:1002C000720E8300F00E700E09008312031341308A
:1002D000C000BD01C101C201C301C401C501C60105
:1002E000C701C801D001D101D301DD01ED012030EA
:1002F000B80083120313B901380884003908840751
:1003000003178D0083160C1483120C08031380004E
:10031000B90A0F303902031D7C294330B2004F3037
:10032000B3004D30B4003930B5003930B6008130FB
:10033000E5002230E6000830E7000030E8008130B8
:10034000E9002130EA000530EB000030EC003230EB
:10035000B000B1012930B800BA01BB01BD01D20122
:10036000831203138501831606309F00D830850061
:1003700000308600EF30870083128316143092001D
:1003800083127D309200831620309900243098002B
:100390008312903098008501FF30DA00FF30DB00D7
:1003A0000000000000000000000000000000DB0B67
:1003B000D029DA0BCE2930308600851400000000E9
:1003C0000000000085101930DA00FF30DB0000006B
:1003D0000000DB0BE729DA0BE529303086008514B5
:1003E00000000000000000008510FF30DA0000006F
:1003F0000000DA0BF7293030860085140000000079
:10040000000000008510FF30DA0000000000DA0B69
:10041000052A38307E2206307E220C307E228B1751
:100420000B1783168C148C168312D21BC02A5118FA
:10043000A02AE51B1E22E91B4E22152A80307E22AF
:1004400065080F39303E8F22660E0F39303E8F22FD
:1004500066080F39303E8F222E308F2267080F3901
:10046000303E8F22680E0F39303E8F2268080F39D8
:10047000303E8F2220308F2241308F2243308F2216
:1004800054308F2249308F2256308F2245308F22B0
:1004900020308F2220308F22E5130800C0307E22CA
:1004A00069080F39303E8F226A0E0F39303E8F2295
:1004B0006A080F39303E8F222E308F226B080F3999
:1004C000303E8F226C0E0F39303E8F226C080F3970
:1004D000303E8F2220308F2253308F2254308F2293
:1004E00041308F224E308F2244308F2242308F2273
:1004F00059308F2220308F22E913080086008510A2
:1005000005110000000085140000000000008510A7
:100510003F30DA0000000000DA0B8A2A080086006B
:100520008510051500000000851400000000000083
:1005300085103F30DA0000000000DA0B9B2A08002B
:10054000D118B32A8516051E152A07160D30D400BA
:100550006030D500840000089900831603130C1640
:100560008312D114152AD408031D152A8316981C4A
:10057000BE2A831207128512D101152A8312152A69
:10058000BD01BB0102308A003A080F39CA3E031888
:100590008A0A82006529DD2ADD2AE12ADA2ADA2A96
:1005A000DA2ADA2ADA2AE62ADA2ADA2ADA2ADA2A1F
:1005B000DA2ADA2ABA01D201152A5114BA01D20173
:1005C000152A4108D000BA01D201152A4108A90014
:1005D0004208AA004308AB004408AC004508AD003F
:1005E0000930D8002930D9000530BE00BA01D20147
:1005F0008B1359088400000803178C000313580854
:1006000003178D0083168C110C1555308D00AA3000
:100610008D008C140C11031383120D1E0D2B0D1263
:10062000D80AD90ABE0BF82AB901BA01BB018B1747
:02063000152A89
:02400E00323F3F
:1042000000000000000000000000000000000000AE
:1042100000004C00430044003000300020005200F9
:104220004400480044002000560031002E003000B9
:04423000300030002A
:00000001FF
